:020000040800F2
:1000000000C00020ED0D0008550800085708000842
:10001000590800085B0800085D080008000000009F
:10002000000000000000000000000000813B00080C
:100030005F08000800000000213C0008653C000843
:10004000350E0008350E0008350E0008350E000884
:10005000350E0008350E0008350E0008350E000874
:10006000350E0008350E0008350E0008350E000864
:10007000350E0008350E0008350E0008350E000854
:10008000350E0008350E0008350E0008350E000844
:10009000350E0008350E0008350E0008350E000834
:1000A000350E0008350E0008350E0008350E000824
:1000B00061080008350E000871080008350E0008B8
:1000C000350E0008350E0008350E0008350E000804
:1000D000350E0008350E000881080008C108000828
:1000E000350E0008350E0008350E0008350E0008E4
:1000F000350E0008350E0008350E0008350E0008D4
:10010000350E0008350E0008350E0008350E0008C3
:10011000350E0008350E0008350E0008350E0008B3
:10012000350E0008350E0008350E0008350E0008A3
:1001300000000000000000000000000000000000BF
:1001400000000000000000000000000000000000AF
:10015000000000000000000000000000000000009F
:10016000000000000000000000000000000000008F
:10017000000000000000000000000000000000007F
:10018000000000000000000000000000000000006F
:10019000000000000000000000000000000000005F
:1001A000000000000000000000000000000000004F
:1001B000000000000000000000000000000000003F
:1001C000000000000000000000000000000000002F
:1001D000000000000000000000000000000000001F
:0401E0005FF8E0F1F3
:1001F000844641EA000313F0030349D1403A23D374
:100200000B6803604B6843608B688360CB68C36096
:100210000B6903614B6943618B698361CB69C3617E
:100220000B6A03624B6A43628B6A8362CB6AC36266
:100230000B6B03634B6B43638B6B8363CB6BC3634E
:1002400040304031403ADBD230320BD30B68036090
:100250004B6843608B688360CB68C360103010319B
:10026000103AF3D20C3205D351F8043B40F8043B6A
:10027000043AF9D2043208D0D2071CBF11F8013B6E
:1002800000F8013B01D30B8803806046704700BF34
:10029000082A13D38B07B1D010F00303AED0C3F1FB
:1002A0000403D21ADB071CBF11F8013B00F8013B25
:1002B000A4D331F8023B20F8023B9FE7043AD9D39C
:1002C000013A11F8013B00F8013BF9D20B780370B9
:1002D0004B7843708B7883706046704738B5002444
:1002E000254600E00134042C0FDC022D0DDC0C4B04
:1002F00003EBC402918853F8340001F021F8002880
:10030000F0D1084B5C550135ECE73DB9054B0022B7
:100310001A7001225A7002229A700325E8B238BD81
:1003200018000020F800002082B002AB03E90300AF
:1003300018B90B685A6302B07047042805D0082822
:1003400007D0019B1B681A64F5E7019B1B689A6341
:10035000F1E7019B1B68DA63EDE7000008B5402177
:10036000054800F0FAFF054801F02EF84FF47A70C6
:1003700003F072F9F3E700BF00080140000100201C
:1003800008B5044A0021044803F0FAF8034B18604A
:1003900008BD00BF245700085D030008FC000020D2
:1003A00030B589B000240494059406940794204B3A
:1003B0009A6942F020029A619A6902F02002009242
:1003C000009A9A6942F004029A619A6902F0040262
:1003D0000192019A9A6942F008029A619A6902F0C0
:1003E00008020292029A9A6942F010029A619B698D
:1003F00003F010030393039B0E4D2246C2212846AF
:1004000000F0A5FFC2230493012305930694022361
:10041000079304A9284600F073FE4FF47E730493FB
:100420000594069404A9044800F06AFE09B030BDA2
:100430000010024000080140000C014008B50748C8
:10044000074B03600523436040F6FF73836000F0B1
:100450008DFF00B908BD00F01BF8FBE7000100208C
:100460000030004010B504460268074B9A4204D0A1
:100470002368B3F1804F03D010BD00F0EFFCF7E725
:10048000024802F0D9FFF7E70008004030010020E1
:1004900072B6FEE700B591B02822002106A805F04B
:1004A000DDF800230193029303930493059309233A
:1004B00006934FF48033079301220A920C92022292
:1004C0000D920E934FF4E0130F9306A800F098FFDF
:1004D00080B90F23019302210291002303934FF46B
:1004E00080620492059301A801F0BCF920B911B013
:1004F0005DF804FBFFF7CCFFFFF7CAFF08B500F07B
:100500009BFCFFF7C7FFFFF74BFF00F0A3FA00F0DB
:10051000FDFA00F08BFB00F0A3FB00F0DBF9FFF726
:100520008DFF00F069FB042000F006F90122802114
:10053000044800F00CFF02F087FFFFF721FF02F0F4
:10054000A1FFFEE7000801400020704710B51E4CD7
:10055000B4F800C0013989B28C18102C2FDCA1EB43
:100560000C0189B29BB1012B25D0002028E0174C4B
:1005700034F811E04FEA1E2E84460CF802EB14F812
:1005800011404470013189B2013A92B26046002AAA
:10059000EDD1184614E084461CF8023B0B4C1B02BC
:1005A00024F811304078034324F81130013189B226
:1005B000013A92B26046002AEDD1002000E001200D
:1005C000034B00221A7010BD2C0100200C010020EA
:1005D000EC02002000B587B0002300930193029342
:1005E000039304930593164A0092164A0192164CFF
:1005F000237060704FF416526260237248252A46B9
:10060000124904F15400FFF7F3FD2A46104904F1A2
:100610000C00FFF7EDFD0F4BC4F8A0300223A4F847
:10062000A430C4F8B0D1204602F0A2FB204602F06C
:10063000FDFB054802F00CFC052003F00DF8F8E77F
:10064000490500084D050008300100208003002006
:100650005804002000080140024B33F810300B8092
:10066000704700BF0C01002080B582B00023ADF8B8
:100670000630ADF8043018E0002439E02A4F00229B
:1006800007EBC40595E80300FFF74EFE57F834105A
:10069000686801F0F9FD0134A642EFDC234800F060
:1006A00093FE4FF4FA7002F0D7FFFFF717FE0646ED
:1006B0000DF106010020FFF7CFFFBDF80630002B3B
:1006C000DAD10024E8E7184B03EBC40553F83410E3
:1006D000686801F05FFDBDF80420154BA3FB0232F2
:1006E00052082832D2B295E80300FFF71DFE01340C
:1006F000A642D3DD0F4B185D013001A9C0B2FFF750
:10070000ABFFBDF80430002BDDD1074F002207EB13
:10071000C40595E80300FFF707FE57F83410686832
:1007200001F0B2FDE3E700BF00000020000100205F
:10073000398EE338F800002010B50146054C2246FA
:10074000054802F01DFF22460021044802F018FF70
:1007500010BD00BF40000020D50500086906000854
:1007600000B583B0114B9A6942F001029A619A690F
:1007700002F001020092009ADA6942F08052DA61D6
:10078000DB6903F080530193019B00220F216FF07E
:10079000010000F087FB064A536823F0E06343F052
:1007A0000073536003B05DF804FB00BF001002400B
:1007B0000000014030B589B00446214BDA6942F0AF
:1007C0000402DA61DB6903F004030193019B02A9CF
:1007D00003A801F023F9069BCBB901F0FFF803460B
:1007E0001848A0FB03239B0C013B1748174A0260E3
:1007F00040F2E732C260436000230361836083619B
:1008000001F030FB054630B1284609B030BD01F09B
:10081000E5F84300E4E70C4801F0E0F9054600285C
:10082000F2D11E2000F076FB0F2C01D90125EBE759
:10083000002221461E2000F035FB054B1C60E3E73B
:100840000010024083DE1B43F0020020000800403D
:100850006C000020FEE7FEE7FEE7FEE7FEE77047DC
:1008600008B5024801F0FAF908BD00BF8003002076
:1008700008B5024801F0F2F908BD00BFF0020020FF
:1008800008B50D4B1B68DB6813F0200F0CD10A4B29
:100890001B68DB6813F0800F0AD1352000F048FB9D
:1008A000054802F019F808BD044802F087FDEEE79C
:1008B000024802F07BFDF0E75804002030010020E0
:1008C00008B5024802F008F808BD00BFA0040020E7
:1008D0007047000000B587B0002302930393049390
:1008E00005930093019315484FF080420260472220
:1008F0004260836040F61F52C2600361836101F071
:10090000B1FA90B94FF48053029302A90B4801F059
:10091000B3FB68B90023009301936946074801F0CF
:10092000F9FC40B907B05DF804FBFFF7B1FDE9E75A
:10093000FFF7AEFDEEE7FFF7ABFDF3E78003002026
:1009400082B003680E4A934204D00E4A93420CD000
:1009500002B070470C4B9A6942F400629A619B693D
:1009600003F400630093009BF2E7074B9A6942F49B
:1009700000529A619B6903F400530193019BE7E7DE
:10098000002C014000340140001002400368B3F124
:10099000804F00D0704700B583B003F50433DA69A7
:1009A00042F00102DA61DB6903F001030193019B6C
:1009B000002205211C2000F075FA1C2000F0AAFA84
:1009C00003B05DF804FB000000B587B0002302937C
:1009D0000393049305930368194A934205D0194A77
:1009E000934217D007B05DF804FB174B9A6942F0A9
:1009F00004029A619B6903F004030093009B4FF487
:100A00008073029302230393059302A90F4800F019
:100A100077FBE7E70C4B9A6942F010029A619B69F9
:100A200003F010030193019B4FF4707302930223B0
:100A30000393059302A9064800F062FBD2E700BFCA
:100A4000002C014000340140001002400008014029
:100A50000010014010B592B0002410941194099434
:100A60000A940B940C940D940E940F94202221461A
:100A700001A804F0F3FD2348234B036047234360A0
:100A8000846040F2F313C36004614461846101F047
:100A900015FA002829D100231093119310A91948A1
:100AA00001F038FC20BB6023099300220A920B92CC
:100AB0000C920D920E920F9209A9124801F062FA5F
:100AC000C8B90023019302930393049305934FF451
:100AD00000520692089301A90A4801F059FC68B92E
:100AE0000848FFF771FF12B010BDFFF7D1FCD2E745
:100AF000FFF7CEFCD7E7FFF7CBFCE2E7FFF7C8FC38
:100B0000EEE700BF38030020002C014010B592B082
:100B100000241094119409940A940B940C940D944D
:100B20000E940F942022214601A804F097FD30482E
:100B3000304B03601F23436084605923C36004610A
:100B40004461846101F0BAF900283CD1002310937C
:100B5000119310A9264801F0DDFB002836D160234F
:100B6000099300220A920B920C920D920E920F9210
:100B700009A91F4801F006FA58BB042209A91C481C
:100B800001F000FA40BB082209A9194801F0FAF95E
:100B900028BB0C2209A9164801F0F4F910BB002368
:100BA000019302930393049305934FF4005206922A
:100BB000089301A90E4801F0EBFBB0B90C48FFF710
:100BC00003FF12B010BDFFF763FCBFE7FFF760FC47
:100BD000C5E7FFF75DFCD0E7FFF75AFCD3E7FFF767
:100BE00057FCD6E7FFF754FCD9E7FFF751FCE5E7E0
:100BF000C80300200034014008B50A480A4B0360CE
:100C00004FF4E133436000238360C36003610C222F
:100C100042618361C36101F0D4FC00B908BDFFF7F4
:100C200037FCFBE7100400200038014008B50A48F3
:100C30000A4B03604FF41653436000238360C36084
:100C400003610C2242618361C36101F0BAFC00B907
:100C500008BDFFF71DFCFBE75804002000440040DE
:100C600008B50A480A4B03604FF4E13343600023A0
:100C70008360C36003610C2242618361C36101F040
:100C8000A0FC00B908BDFFF703FCFBE7A0040020AF
:100C90000048004030B58BB00023069307930893BB
:100CA000099303684B4A934207D04B4A93422ED094
:100CB0004A4A93425BD00BB030BD494B9A6942F42B
:100CC00080429A619A6902F480420092009A9A697D
:100CD00042F004029A619B6903F004030193019BB3
:100CE0004FF40073069302230793032309933D4CAB
:100CF00006A9204600F004FA4FF48063069300230F
:100D00000793089306A9204600F0FAF9D3E7344B7D
:100D1000DA6942F40032DA61DA6902F400320292EE
:100D2000029A9A6942F004029A619B6903F00403F3
:100D30000393039B0423069302230793032309933E
:100D4000284D06A9284600F0DBF908230693002465
:100D50000794089406A9284600F0D2F922460521F6
:100D6000262000F09FF8262000F0D4F8A3E71C4BC3
:100D7000DA6942F48022DA61DA6902F480220492AC
:100D8000049A9A6942F008029A619B6903F0080389
:100D90000593059B4FF48063069302230793032377
:100DA0000993114D06A9284600F0AAF94FF40063F3
:100DB000069300240794089406A9284600F0A0F999
:100DC00022460521272000F06DF8272000F0A2F828
:100DD00071E700BF00380140004400400048004077
:100DE0000010024000080140000C0140FFF770FDB8
:100DF0000B480C490C4A002302E0D458C450043379
:100E0000C4188C42F9D3094A094C002301E013604D
:100E10000432A242FBD304F0FDFBFFF76FFB7047E7
:100E200000000020F800002098590008F800002079
:100E3000881E0020FEE7000008B5074A136843F04B
:100E400010031360032000F01BF80F20FFF7B2FC23
:100E5000FFF786FC002008BD00200240034A11680D
:100E6000034B1B780B441360704700BFE80400205D
:100E700068000020014B1868704700BFE80400209C
:100E8000074AD36823F4E0631B041B0C000200F440
:100E9000E060034343F0BF6343F40033D360704723
:100EA00000ED00E000B5194BDB68C3F30223C3F18A
:100EB000070CBCF1040F28BF4FF0040C03F1040E23
:100EC000BEF1060F18D9033B4FF0FF3E0EFA0CFCA3
:100ED00021EA0C0199400EFA03F322EA03031943B5
:100EE00000280BDB0901C9B200F1604000F5614048
:100EF00080F800135DF804FB0023E5E700F00F0025
:100F00000901C9B2024B1954F4E700BF00ED00E03B
:100F100014ED00E0002807DB00F01F024009012368
:100F20009340024A42F82030704700BF00E100E0E1
:100F3000002808DB00F01F024009012393406030C5
:100F4000014A42F82030704700E100E090F821307B
:100F5000DBB2022B06D004238363002380F8203009
:100F6000012070470268136823F00E0313600268C3
:100F7000136823F001031360036CC16B012202FAB2
:100F800003F34B6080F82120002380F820301846BE
:100F90007047000008B590F82130DBB2022B03D077
:100FA00004238363012008BD0268136823F00E0345
:100FB00013600268136823F00103136003684C4A4E
:100FC00093424ED9783A934224D01432934230D08F
:100FD000143293422FD0143293422FD014329342C2
:100FE0002FD0143293422FD0143293422FD002F5D7
:100FF000627293422ED0143293422DD01432934217
:101000002CD01432934202D04FF4803203E04FF4DC
:10101000805200E00122374B5A60012380F82130D2
:10102000002380F82030436B002B5ED098470020CF
:10103000B9E71022EFE74FF48072ECE74FF48052EB
:10104000E9E74FF48032E6E74FF48012E3E74FF030
:101050008072E0E70122DEE71022DCE74FF48072C5
:10106000D9E7254A934224D01432934225D0143232
:10107000934224D01432934224D01432934224D089
:101080001432934224D01432934224D002F5627277
:10109000934223D01432934222D01432934221D06F
:1010A0001432934202D04FF4803203E04FF4805266
:1010B00000E00122114B5A60AFE71022FAE74FF42B
:1010C0008072F7E74FF48052F4E74FF48032F1E793
:1010D0004FF48012EEE74FF08072EBE70122E9E770
:1010E0001022E7E74FF48072E4E700205BE700BFDF
:1010F000800002400004024008000240000002405C
:1011000070B582B00024A446B0E0874DAA4210D04A
:1011100007D9864DAA420CD005F58035AA4208D0E1
:1011200013E0A5F58015AA4203D005F57025AA4263
:1011300007D18A68002A62D0012A5BD04361082463
:1011400003E0A5F58015AA42F3D0BEF1FF0F58D8F1
:101150000646BEF1FF0F56D84FEA8C0233680F25C2
:10116000954023EA050304FA02F2134333604B6807
:1011700013F0805F78D06E4B9A6942F001029A6159
:101180009B6903F001030193019B4FEA9C02951CAC
:10119000684B53F825600CF003039D000F23AB4010
:1011A00026EA0306644B984233D003F580639842E5
:1011B00000F0988003F58063984200F0958003F575
:1011C0008063984200F0928003F58063984200F0BB
:1011D0008F8003F58063984219D006231AE0CC680B
:1011E000B3E7CC680434B0E7CC680834ADE7CC682A
:1011F0000C34AAE703610824A7E70024A5E7042428
:10120000A3E7061DA5E7ACF108029200A6E70523B7
:1012100000E00023AB4033430232464D45F8223014
:101220004B6813F4801F65D0444A936843EA0E0369
:1012300093604B6813F4001F62D0404AD36843EABE
:101240000E03D3604B6813F4003F5FD03B4A5368F2
:1012500043EA0E0353604B6813F4803F5CD0374A77
:10126000136843EA0E0313600CF1010C0A6832FAAA
:101270000CF357D0012303FA0CF302EA030E33EA0E
:101280000202F1D14A68122A3FF63FAF122A3FF616
:101290005CAF01A555F822F033110008DF110008FA
:1012A000E9110008FB1100084B1100084B11000860
:1012B0004B1100084B1100084B1100084B1100089E
:1012C0004B1100084B1100084B1100084B1100088E
:1012D0004B1100084B1100084B110008E3110008E6
:1012E000EF110008012395E7022393E7032391E719
:1012F00004238FE7114A936823EA0E03936098E76B
:101300000E4AD36823EA0E03D3609BE70B4A536867
:1013100023EA0E0353609EE7084A136823EA0E038C
:101320001360A1E702B070BD000022100000311070
:10133000001002400000014000080140000401408C
:101340008368194201D001207047002070470AB11C
:1013500001617047090401617047C36801EA030233
:1013600021EA030141EA02410161704750B338B5F7
:10137000044603684CF6CC421A60036845F25552A5
:101380001A60036842685A60036882689A60FFF7CF
:1013900071FD05462368DA6812F0030F0DD0FFF7E0
:1013A00069FD401B41F23C339842F3D92368DB6866
:1013B00013F0030FEED0032003E04AF6AA221A60CE
:1013C000002038BD0120704703684AF6AA221A603F
:1013D0000020704782B0084B1B68084AA2FB032319
:1013E0005B0A00FB03F3019300BF019B5A1E0192AD
:1013F000002BF9D102B0704764000020D34D621079
:10140000002800F0F18170B582B00446036813F043
:10141000010F2CD0994B5B6803F00C03042B1DD0FB
:10142000964B5B6803F00C03082B12D06368B3F58E
:10143000803F41D0002B55D103F1804303F50433A5
:101440001A6822F480321A601A6822F480221A6024
:1014500037E08A4B5B6813F4803FE7D0874B1B680B
:1014600013F4003F03D06368002B00F0BF812368B2
:1014700013F0020F75D0814B5B6813F00C0F5FD037
:101480007E4B5B6803F00C03082B54D02369002BC0
:1014900000F08A807A4B01221A60FFF7EBFC0546C8
:1014A000764B1B6813F0020F75D1FFF7E3FC401B6E
:1014B0000228F5D903209EE1704A136843F4803373
:1014C0001360636843B3FFF7D5FC05466B4B1B689D
:1014D00013F4003FCBD1FFF7CDFC401B6428F5D9B6
:1014E000032088E1B3F5A02F09D0644B1A6822F4D9
:1014F00080321A601A6822F480221A60E1E703F150
:101500008043A3F53C331A6842F480221A601A68BB
:1015100042F480321A60D4E7FFF7ACFC0546574B23
:101520001B6813F4003FA2D0FFF7A4FC401B642803
:10153000F5D903205FE1514B5B6813F4803FA5D1DF
:101540004E4B1B6813F0020F03D02369012B40F0B0
:101550004F814A4A136823F0F803616943EAC103E3
:101560001360236813F0080F33D0A369002B5CD0FD
:10157000434B0122C3F88024FFF77CFC05463F4B18
:101580005B6A13F0020F21D1FFF774FC401B0228A5
:10159000F5D903202FE1394A136823F0F803616974
:1015A00043EAC1031360DCE7354B00221A60FFF702
:1015B00061FC0546314B1B6813F0020FD1D0FFF7D9
:1015C00059FC401B0228F5D9032014E10120FFF744
:1015D00001FF236813F0040F00F09680274BDB69AE
:1015E00013F0805F34D1254BDA6942F08052DA6122
:1015F000DB6903F080530193019B0125214B1B689C
:1016000013F4807F26D0E368012B3DD0002B53D10B
:1016100003F1804303F504331A6A22F001021A62CF
:101620001A6A22F004021A6233E0154B0022C3F852
:101630008024FFF71FFC0546104B5B6A13F0020F76
:10164000C7D0FFF717FC401B0228F5D90320D2E0D2
:101650000025D3E70B4A136843F480731360FFF748
:1016600009FC0646074B1B6813F4807FCBD1FFF7BC
:1016700001FC801B6428F5D90320BCE00010024067
:1016800000004242007000405F4A136A43F00103C9
:101690001362E36833B3FFF7EDFB06465A4B1B6A50
:1016A00013F0020F2FD1FFF7E5FB801B41F28833C7
:1016B0009842F3D903209EE0052B09D0524B1A6AB9
:1016C00022F001021A621A6A22F004021A62E0E7AA
:1016D0004D4B1A6A42F004021A621A6A42F0010281
:1016E0001A62D6E7FFF7C6FB0646474B1B6A13F0A4
:1016F000020F08D0FFF7BEFB801B41F288339842EF
:10170000F3D9032077E0E5B9E369002B72D03E4AB4
:10171000526802F00C02082A56D0022B17D03B4B1D
:1017200000221A66FFF7A6FB0446374B1B6813F02E
:10173000007F47D0FFF79EFB001B0228F5D903204E
:1017400059E0314AD36923F08053D361DCE72F4B52
:1017500000221A66FFF78EFB05462B4B1B6813F021
:10176000007F06D0FFF786FB401B0228F5D9032037
:1017700041E0236AB3F5803F1AD023494B6823F434
:101780007413226A606A024313434B601F4B0122A9
:101790001A66FFF76FFB04461B4B1B6813F0007FB4
:1017A0000ED1FFF767FB001B0228F5D9032022E0CA
:1017B000154A536823F40033A1680B435360DCE7F8
:1017C000002018E0002016E0012B16D00E4B5B68BD
:1017D00003F48031226A914211D103F47013626ADA
:1017E00093420ED1002006E001207047012002E064
:1017F000012000E0002002B070BD0120FBE70120C5
:10180000F9E70120F7E700BF001002400000424264
:101810000F4B5B6803F00C02082A01D00D4870479B
:10182000C3F383420C49885C13F4803F0BD0084B10
:101830005B68C3F34043094AD35C064A02FB00F0ED
:10184000B0FBF3F07047064B03FB00F0704700BF9E
:101850000010024000127A006C5700087C57000804
:1018600000093D00002800F0A08070B50D46044638
:10187000524B1B6803F007038B420BD24F4A13688D
:1018800023F007030B431360136803F007038B4235
:1018900040F08D80236813F0020F17D013F0040F6F
:1018A00004D0474A536843F4E0635360236813F05D
:1018B000080F04D0424A536843F460535360404ACF
:1018C000536823F0F003A1680B435360236813F0BF
:1018D000010F31D06368012B20D0022B25D0384A6C
:1018E000126812F0020F64D035494A6822F00302F0
:1018F00013434B60FFF7BEFA0646314B5B6803F0BB
:101900000C036268B3EB820F16D0FFF7B3FA801BAB
:1019100041F288339842F0D9032045E0284A126802
:1019200012F4003FE0D101203EE0254A126812F097
:10193000007FD9D1012037E0204B1B6803F007035B
:10194000AB420AD91D4A136823F007032B431360E7
:10195000136803F00703AB422DD1236813F0040F83
:1019600006D0174A536823F4E063E1680B435360E1
:10197000236813F0080F07D0114A536823F460530B
:10198000216943EAC1035360FFF742FF0C4B5B68D8
:10199000C3F303130B4AD35CD8400B4B18600B4BBB
:1019A0001868FEF707FF002070BD01207047012076
:1019B000FAE70120F8E70120F6E700BF0020024027
:1019C0000010024054570008640000206C00002002
:1019D000014B1868704700BF6400002008B5FFF78E
:1019E000F7FF044B5B68C3F30223034AD35CD84080
:1019F00008BD00BF001002406457000808B5FFF79B
:101A0000E7FF044B5B68C3F3C223034AD35CD840AF
:101A100008BD00BF00100240645700080F23036098
:101A20000B4B5A6802F0030242605A6802F0F0025F
:101A300082605A6802F4E062C2605B68DB0803F40B
:101A4000E0630361034B1B6803F007030B607047FF
:101A5000001002400020024030B4036A026A22F003
:101A6000010202624268846924F073040D682C4309
:101A700023F0020C8B6843EA0C03104DA84203D0FC
:101A800005F50065A84205D123F00803CD682B4376
:101A900023F00403094DA84203D005F50065A842D0
:101AA00005D122F440724D692A438D692A43426070
:101AB00084614A684263036230BC7047002C014075
:101AC00030B4036A026A22F4807202624268C46916
:101AD00024F0730C0C6844EA0C0523F400738C6842
:101AE00043EA0423114CA04203D004F50064A04251
:101AF00006D123F40063CC6843EA042323F4806313
:101B00000A4CA04203D004F50064A04207D122F49D
:101B100040524C6942EA04128C6942EA0412426063
:101B2000C5614A68C263036230BC7047002C014043
:101B300030B4036A026A22F4805202624468C269C5
:101B400022F4E6420D6842EA052223F400538D6830
:101B500043EA0533094DA84203D005F50065A842C4
:101B600004D124F480444D6944EA85144460C26180
:101B70004A680264036230BC704700BF002C014019
:101B800010B4036A046A24F001040462846924F036
:101B9000F00C4CEA021223F00A030B438261036249
:101BA00010BC704710B4036A046A24F01004046285
:101BB000846924F4704C4CEA023223F0A00343EA17
:101BC00001138261036210BC7047836823F07003C5
:101BD0000B4343F0070383607047000090F83D30EB
:101BE000DBB2012B2FD1022380F83D300268D3688D
:101BF00043F00103D3600368154A934218D002F5FD
:101C00000062934214D0B3F1804F11D0A2F5983204
:101C100093420DD002F58062934209D002F58062B2
:101C2000934205D01A6842F001021A600020704702
:101C30009A6802F00702062A07D01A6842F00102E9
:101C40001A6000207047012070470020704700BFD5
:101C5000002C0140704770477047704770B50446CC
:101C60000368DE681D6915F0020F10D016F0020F30
:101C70000DD06FF002021A610123037703689B699C
:101C800013F0030F5ED0FFF7E6FF0023237715F074
:101C9000040F12D016F0040F0FD023686FF0040267
:101CA0001A610223237723689B6913F4407F4FD086
:101CB0002046FFF7D0FF0023237715F0080F12D03E
:101CC00016F0080F0FD023686FF008021A61042382
:101CD00023772368DB6913F0030F40D02046FFF71A
:101CE000BAFF0023237715F0100F12D016F0100F53
:101CF0000FD023686FF010021A610823237723683E
:101D0000DB6913F4407F31D02046FFF7A4FF0023A6
:101D1000237715F0010F02D016F0010F2DD115F029
:101D2000800F02D016F0800F2FD115F0400F02D097
:101D300016F0400F31D115F0200F02D016F0200F11
:101D400033D170BDFFF786FF2046FFF785FF9CE784
:101D50002046FFF77FFF2046FFF77EFFABE72046D8
:101D6000FFF778FF2046FFF777FFBAE72046FFF737
:101D700071FF2046FFF770FFC9E723686FF001028B
:101D80001A612046FEF76EFBC9E723686FF08002F8
:101D90001A61204600F026FBC7E723686FF0400277
:101DA0001A612046FFF759FFC5E723686FF020024C
:101DB0001A61204600F015FBC3E700000368284ABB
:101DC000904212D002F5006290420ED0B0F1804FE6
:101DD0000BD0A2F59832904207D002F58062904273
:101DE00003D002F58062904203D123F070034A6869
:101DF00013431B4A904212D002F5006290420ED06B
:101E0000B0F1804F0BD0A2F59832904207D002F586
:101E10008062904203D002F58062904203D123F4A5
:101E20004073CA68134323F080034A691343036075
:101E30008B68C3620B688362094B984203D003F539
:101E40000063984201D10B69036301234361036975
:101E500013F0010F03D0036923F0010303617047FE
:101E6000002C014040B310B5044690F83D30F3B16A
:101E7000022384F83D30214651F8040BFFF79EFF02
:101E8000012384F8463084F83E3084F83F3084F8EB
:101E9000403084F8413084F8423084F8433084F88C
:101EA000443084F8453084F83D30002010BD80F87F
:101EB0003C30FEF76BFDDBE70120704740B310B507
:101EC000044690F83D30F3B1022384F83D302146BA
:101ED00051F8040BFFF772FF012384F8463084F8B1
:101EE0003E3084F83F3084F8403084F8413084F844
:101EF000423084F8433084F8443084F8453084F824
:101F00003D30002010BD80F83C30FEF719FDDBE7C6
:101F10000120704730B4036A026A22F010020262A4
:101F20004468826922F4E6420D6842EA052223F001
:101F300020038D6843EA0513114DA84203D005F52F
:101F40000065A84206D123F08003CD6843EA05135B
:101F500023F040030A4DA84203D005F50065A842CE
:101F600007D124F440644D6944EA85048D6944EA4C
:101F70008504446082614A688263036230BC7047B2
:101F8000002C014038B590F83C30012B66D0044657
:101F90000D46012380F83C300C2A5AD8DFE802F0C5
:101FA000075959591B595959305959594400006812
:101FB000FFF752FD2268936943F00803936122689A
:101FC000936923F0040393612268936929690B43A1
:101FD000936100203EE00068FFF79CFF2268936950
:101FE00043F4006393612268936923F480639361EF
:101FF00022689369296943EA01239361002029E05B
:102000000068FFF75DFD2268D36943F00803D361E0
:102010002268D36923F00403D3612268D369296954
:102020000B43D361002015E00068FFF781FD2268B3
:10203000D36943F40063D3612268D36923F48063D6
:10204000D3612268D369296943EA0123D36100205F
:1020500000E00120002384F83C3038BD0220FCE77A
:1020600010B4846824F47F4C42EA03220A4342EA13
:102070000C02826010BC704790F83C30012B78D085
:1020800010B50446012380F83C30022380F83D302F
:102090000268936823F47F4323F0770393600B680F
:1020A000602B4CD029D8402B54D00CD9502B22D1A6
:1020B000CA6849680068FFF763FD50212068FFF790
:1020C00084FD002005E0202B0DD009D9302B0AD04B
:1020D0000120012384F83D30002384F83C3010BDFA
:1020E0000BB1102B05D119462068FFF76EFD0020BB
:1020F000EFE70120EDE70120EBE7B3F5805F34D097
:10210000B3F5005F0CD1CB684A6889680068FFF7B7
:10211000A7FF2268936843F4804393600020D8E7C8
:10212000702B24D1CB684A6889680068FFF798FF54
:102130002268936843F0770393600020C9E7CA6878
:1021400049680068FFF72EFD60212068FFF73DFD1C
:102150000020BEE7CA6849680068FFF711FD40210A
:102160002068FFF732FD0020B3E70020B1E701202F
:10217000AFE70220704701F01F01012303FA01FCC1
:10218000036A23EA0C030362036A02FA01F10B43B8
:102190000362704710B50446084600293AD194F806
:1021A0003E30DBB2013B18BF0123002B66D1002873
:1021B00049D1022384F83E30012201462068FFF70E
:1021C000DAFF23682F4A934203D002F5006293425C
:1021D00003D15A6C42F400425A642368294A93425C
:1021E00041D002F5006293423DD0B3F1804F3AD026
:1021F000A2F59832934236D002F58062934232D0F3
:1022000002F5806293422ED01A6842F001021A60F1
:10221000002032E0042908D008290DD094F841307C
:10222000DBB2013B18BF0123BFE794F83F30DBB2BC
:10223000013B18BF0123B8E794F84030DBB2013B03
:1022400018BF0123B1E7042805D0082807D00223CE
:1022500084F84130B0E7022384F83F30ACE7022332
:1022600084F84030A8E79A6802F00702062A07D0EF
:102270001A6842F001021A60002010BD0120FCE73C
:102280000020FAE7002C014038B504460D46002234
:102290000068FFF770FF23681D4A934218D002F5CB
:1022A0000062934214D02368196A41F2111211425C
:1022B00008D1196A40F24442114203D11A6822F04F
:1022C00001021A609DB9012384F83E30002038BD18
:1022D000196A41F211121142E5D1196A40F24442E1
:1022E0001142E0D15A6C22F400425A64DBE7042D1B
:1022F00005D0082D07D0012384F84130E6E70123FB
:1023000084F83F30E2E7012384F84030DEE700BF85
:10231000002C014090F83C30012B34D010B4012344
:1023200080F83C30022380F83D3003685A689C688E
:1023300022F0700C0A6842EA0C025A600368134AE1
:10234000934212D002F5006293420ED0B3F1804F57
:102350000BD0A2F59832934207D002F580629342E7
:1023600003D002F58062934204D124F080044A68CD
:1023700014439C60012380F83D30002380F83C30FA
:10238000184610BC70470220704700BF002C014067
:1023900090F83C30012B22D0012380F83C30CB68F0
:1023A00023F440738A68134323F480634A68134319
:1023B00023F400630A68134323F480530A69134328
:1023C00023F400534A69134323F48043CA69134337
:1023D00002685364002380F83C301846704702209E
:1023E000704770477047026802F10C0353E8003FE2
:1023F00023F490730C3242E800310029F3D10268D3
:1024000002F1140353E8003F23F00103143242E8C1
:1024100000310029F3D1036B012B05D0202380F874
:102420004230002303637047026802F10C0353E853
:10243000003F23F010030C3242E800310029F3D1B1
:10244000ECE790F84130DBB2212B01D0022070473D
:102450008368B3F5805F17D0036A5A1C02621A784A
:1024600003685A60C38C9BB2013B9BB2C3844BB9D7
:102470000268D36823F08003D3600268D36843F016
:102480004003D360002070470369002BE4D1036A46
:102490001B880268C3F308035360036A02330362B4
:1024A000E0E7000010B504460268136923F44053C6
:1024B000C1680B43136183680269134342691A437D
:1024C0000168CB6823F4B05323F00C031343CB60B3
:1024D0000268536923F4407381690B4353610268B6
:1024E000134B9A4220D0FFF779FA024602EB8202A0
:1024F00002EB820263689B00B2FBF3F20D48A0FB83
:1025000002314909642303FB11231B013233A0FB71
:1025100003235B0903F0F00202EB011203F00F0347
:10252000216813448B6010BDFFF768FA0246DDE7AF
:10253000003801401F85EB512DE9F04383B005467B
:102540000E4617469946DDF828802C68246836EA3E
:1025500004030CBF4FF0010C4FF0000CBC4528D118
:10256000B8F1FF3FF1D0FEF785FCA0EB0900404534
:1025700023D8B8F1000F22D02B68DA6812F0040FCC
:10258000E3D0802EE1D0402EDFD01A6812F0080F81
:10259000DBD0002401941A6801925B680193019BCF
:1025A0002846FFF720FF08236B6485F84040012090
:1025B00000E0002003B0BDE8F0830320FAE7032029
:1025C000F8E760B310B5044690F8413013B3242304
:1025D00084F841302268D36823F40053D360204646
:1025E000FFF760FF2268136923F4904313612268A8
:1025F000536923F02A0353612268D36843F40053DC
:10260000D36000206064202384F8413084F8423095
:10261000606310BD80F84030FEF73CFBD7E7012037
:1026200070472DE9F04182B01E4690F84130DBB290
:10263000202B56D104460D469046002955D00AB9A4
:1026400001204FE000234364212380F84130FEF74E
:1026500011FC0746A4F82480A4F82680A368B3F5EB
:10266000805F02D04FF0000814E023692BB34FF0D5
:1026700000080FE0202384F84130032032E038F8CE
:10268000023B2268C3F308035360E28C92B2013A22
:1026900092B2E284E38C9BB293B100963B46002257
:1026A00080212046FFF748FF0028E3D1002DE6D027
:1026B00015F8012B23685A60E7E7A8460025E9E7EB
:1026C00000963B46002240212046FFF735FF18B90F
:1026D000202384F8413005E0202384F84130032092
:1026E00000E0022002B0BDE8F0810120FAE72DE908
:1026F000F04182B01E4690F84230DBB2202B59D117
:1027000004460D469046002958D00AB9012052E0EF
:1027100000234364222280F842200363FEF7AAFBD1
:102720000746A4F82C80A4F82E80A368B3F5805F38
:1027300002D04FF000081CE0236913B14FF00008ED
:1027400017E0A846002514E0202384F84230032037
:1027500031E023685B68C3F3080328F8023B03E019
:1027600023685B682B700135E28D92B2013A92B218
:10277000E285E38D9BB2C3B100963B460022202147
:102780002046FFF7D9FE0028DED1002DE1D0A36856
:10279000B3F5805FE4D013B92369002BE0D0236840
:1027A0005B6803F07F032B70DDE7202384F8423061
:1027B000002000E0022002B0BDE8F0810120FAE72D
:1027C000704708B50168CA6822F04002CA6020223A
:1027D00080F84120FFF7F4FF002008BD70477047E4
:1027E00008B5406A0023C385C384FFF7F8FF08BD1E
:1027F000704790F84230DBB2222B69D18368B3F581
:10280000805F4FD0826AB3F5805F04D0002B56D131
:102810000369002B53D103685B681370836A01332B
:102820008362C38D9BB2013B9BB2C385002B51D108
:1028300000B583B00268D36823F02003D360026838
:10284000D36823F48073D3600268536923F00103D3
:102850005361202380F8423000234363036B012B34
:1028600033D100230363026802F10C0353E8003FF5
:1028700023F010030C3242E800310029F3D1036841
:102880001A6812F0100F06D0002201921A68019205
:102890005B680193019B818DFFF7AAFF002003B0C5
:1028A0005DF804FB0269002AACD1826A03685B68A8
:1028B000C3F308031380836A02338362B1E70368BA
:1028C0005B6803F07F031370A8E7FFF787FFE5E776
:1028D000022070470020704730B583B0044602687C
:1028E0001368D068516913F00F0505D113F0200F5C
:1028F00002D010F0200F19D12DB111F0010119D122
:1029000010F4907F16D1216B01297DD013F0800F38
:1029100003D010F0800F40F0188113F0400F03D067
:1029200010F0400F40F0158103B030BD2046FFF796
:1029300060FFF9E713F0010F06D010F4807F03D099
:10294000626C42F00102626413F0040F04D019B10A
:10295000626C42F00202626413F0020F04D019B1FB
:10296000626C42F00402626413F0080F07D010F0AA
:10297000200F00D119B1626C42F008026264626CEF
:10298000002AD1D013F0200F02D010F0200F29D14F
:1029900023685B6903F04003626C12F0080F00D1FA
:1029A00063B32046FFF71FFD23685B6913F0400FF8
:1029B00020D0226802F1140353E8003F23F04003C3
:1029C000143242E800310029F3D1E36B73B1634A5A
:1029D0005A63E06BFEF7DEFA0028A5D0E06B436B8C
:1029E0009847A1E72046FFF704FFD1E72046FFF70D
:1029F000F6FE99E72046FFF7F2FE95E72046FFF73F
:102A0000EEFE002363648FE713F0100F3FF47EAFF8
:102A100010F0100F3FF47AAF002301931368019375
:102A200053680193019B536913F0400F51D0E26B3F
:102A300013685B689BB2002B3FF476AFA18D99427F
:102A40007FF672AFE3859369202B37D0226802F1BD
:102A50000C0353E8003F23F480730C3242E800314A
:102A60000029F3D1226802F1140353E8003F23F058
:102A70000103143242E800310029F3D1226802F147
:102A8000140353E8003F23F04003143242E80031BE
:102A90000029F3D1202384F84230002323632268E5
:102AA00002F10C0353E8003F23F010030C3242E81C
:102AB00000310029F3D1E06BFEF748FA022363638B
:102AC000A18DE38D9BB2C91A89B22046FFF790FE13
:102AD0002AE7A18DE38D9BB2C91A89B2E38D9BB21F
:102AE000002B3FF421AF00293FF41EAF226802F112
:102AF0000C0353E8003F23F490730C3242E800309B
:102B00000028F3D1226802F1140353E8003F23F0B8
:102B10000103143242E800300028F3D1202384F866
:102B2000423000232363226802F10C0353E8003F84
:102B300023F010030C3242E800300028F3D10223C6
:102B400063632046FFF754FEEEE62046FFF779FC6C
:102B5000EAE62046FFF735FEE6E600BFE12700087B
:102B600008B5D0F8B0315B69481C0146984700B9F8
:102B700008BD00F0F1F8FBE71388052B01D0032016
:102B8000704710B58C464B78897841EA03210131B2
:102B9000D0F8B0315C6801231A4689B20CF1030009
:102BA000A04700B910BD00F0D7F8FBE738B513888F
:102BB000052B27D98C4614464B78897841EA0321A6
:102BC000013189B29CF803309CF8042042EA0322C8
:102BD0009CF805E0531E9BB2772B15D85300DBB24F
:102BE000734501D003200EE0D0F8B0315D680123B9
:102BF0000CF10600A84710B90523238003E000F07C
:102C0000ABF800E0032038BD0320FCE71388052B58
:102C100001D00320704770B58C4614464B788978F4
:102C200041EA0321013189B29CF803309CF8045039
:102C300045EA03256B1E9BB27C2B1DD80023138015
:102C4000E64603220EF8022B2288013222806A0017
:102C50008CF80120228801322280D0F8B0215668F9
:102C60002A467046B04720B9238803EB45052580E6
:102C700070BD00F071F8FBE70320F9E72DE9F84398
:102C80001388092B4DD907460C4615464B788E788C
:102C900046EA03260136B6B2CB7891F8048048EABA
:102CA00003284B79897941EA0321013189B2E3791B
:102CB000227A42EA0322607A08F1FF339BB27C2B2E
:102CC00032D89AB3792A33D8B0EB420F01D003201F
:102CD00028E0D7F8B031D3F80490012304F10A00BA
:102CE000C8470346C8B928802046172200F8022B9F
:102CF0002A8801322A804FEA480262702A8801320B
:102D00002A80D7F8B021546842463146A04720B9FE
:102D10002B8803EB4808A5F8008018B100F01CF8D8
:102D200000E00020BDE8F8830320FBE70320F9E77B
:102D30000320F7E738B508461546054B1C882246A0
:102D400004490130FDF754FA01342C80002038BDCD
:102D50000C050020EC040020012805D0072805D030
:102D600008B1042070477047022070470620704762
:102D700038B54278531EDBB2F62B2DD80446194BDA
:102D80001A7003780BB1022527E0174B174A1A6017
:102D9000174B184A1A60184B184A1A60184B194AF0
:102DA0001A60194B00221A60184B194A1A60194B05
:102DB000194A1A60194B1A4A1A6000F0E3F80546DE
:102DC00058B9204600F04AFA48B12278154B1A70DB
:102DD000154B01221A7000E00225284638BD032554
:102DE000FBE700BF310500201C050020FD2F000877
:102DF000200500201F300008140500208B3000083B
:102E0000100500203D300008180500202405002092
:102E10001931000828050020AB3100082C050020DE
:102E2000053200080F0500207000002008B5064B91
:102E30001B78012B01D0062008BD044B1B68984766
:102E40000020014B1870F7E7700000201C050020DF
:102E500070B582B0364B1D78002D65D104460DF15A
:102E6000070100F011FA012802D0284602B070BD17
:102E70009DF80730022B14D0042BF6D1D4F8B411EE
:102E800008782C4B18702C4B01221A7000230F2B42
:102E900029DC2A4A12F833202AB3904219D0013390
:102EA000F5E7274B1E68234604F5DD7204F5DA7159
:102EB0002448B04706460028D7D16278214B1B78BA
:102EC0009A4200D093BB0421204600F0D2F9354647
:102ED000CBE71A4A02EBC3035B6804F5DD722046B8
:102EE0009847154B1870144B1B78A3B10022A4F817
:102EF000BA21104A1278D4F8B4110120A4F8BA010A
:102F000042F080020A70D4F8B411B4F8BA21101853
:102F1000A4F8BA018B540C4B1B68B4F8BA21D4F84E
:102F2000B41120469847A0E706259EE705469CE792
:102F300070000020300500200E05002074000020E5
:102F400010050020320500201405002000B5FF22E6
:102F500096460AE010F8013B5340084AD25C82EAE8
:102F60000E02074911F803E061464B1E1FFA83FC6D
:102F70000029EFD142EA0E205DF804FB80570008DB
:102F80008058000830B591B0044600F057F920464B
:102F900000F09EF9012805D0032400F057F92046DF
:102FA00011B030BD6368B3F5964F20D85B00124D69
:102FB000B5FBF3F5EC4604F1600EBEE80F00ACE89B
:102FC0000F00BEE80F00ACE80F00BEE80F00ACE851
:102FD0000F009EE807008CE80700543494E80E00C8
:102FE000A8B200F0F3F9012803D00324D5E7232584
:102FF000E0E70024D1E700BFA07F170010B504462A
:1030000000F01CF9002284F8A7200121204600F0DE
:1030100097F9204600F0E1F900F018F910BD10B55D
:10302000044600F00BF900221146204600F088F912
:10303000204600F0E4F900F009F910BDF8B50746A4
:103040000D4616461C4600F0F9F8B4F8AE319BB2B6
:10305000032B04D8052400F0F9F82046F8BDB4F895
:10306000AE1189B204F1A800FFF770FF58B994F8C7
:10307000A8303B70B4F8AE319BB2033B3380A93427
:103080002C600024E7E70524E5E7F8B504460E4682
:10309000174600F0D3F894F8A730DBB2012B04D028
:1030A000052400F0D3F82046F8BD731EC4F8A831FB
:1030B0000125A4F8AC51637806F8013CB4F8AC31B2
:1030C0009BB2DA1992B2A4F8AC21B4F8AC1189B26F
:1030D000D4F8A801FFF73AFFB4F8AC319BB25A1903
:1030E00092B2A4F8AC21C2B2234483F8A820B4F869
:1030F000AC319BB25A1992B2A4F8AC21C0F30720AC
:10310000234483F8A80084F8A6502A4600212046CC
:1031100000F016F90024C4E710B582B004460DF1A2
:10312000070100F038F994F8A730DBB2032B06D87A
:10313000DFE803F0020C2208204600F04EF90020E0
:1031400002B010BD204600F048F9F8E70023A4F8CB
:10315000AE31B4F8AE319BB25A1C92B2A4F8AE2193
:103160009DF80720234483F8A820022384F8A73081
:10317000204600F032F9E2E7B4F8AE319BB2FF2B03
:103180000FD8B4F8AE319BB25A1C92B2A4F8AE215B
:103190009DF80720234483F8A820204600F01DF95D
:1031A000CDE7032384F8A730F7E738B5044690F855
:1031B000A63003F0FF0523B1012D07D000252846D6
:1031C00038BD0022012100F0BBF8F8E7B0F8AC31BF
:1031D0009BB253B1B0F8AC2192B2D0F8A81100F074
:1031E000CFF80025A4F8AC51E9E7082100F041F838
:1031F000054600220121204600F0A2F8002384F8B1
:10320000A630DCE738B5044690F8A73063B103F088
:10321000FF02022A0DD00025204600F0F0F801231D
:1032200084F8A730284638BD012100F022F8054671
:10323000F2E7022100F01DF80546EDE708B500F0C1
:1032400045F9014B186008BD3405002008B5024B54
:10325000186800F05FF908BD3405002010B5044679
:10326000002000F017FAC4F89C00003818BF0120B5
:1032700010BDD0F89C0028B108B500F03BFAC0435F
:10328000C00F08BD0020704710B50C464FF0FF334B
:1032900000220F21D0F89C0000F06AFA01380728BC
:1032A00014D8DFE800F00407130B1313130F0120E9
:1032B00020700CE002232370012008E00423237017
:1032C000012004E008232370012000E0002010BD4D
:1032D00008B543680361002343618361037A012BCE
:1032E00010D0022B12D00BB1002008BDC3610C23FB
:1032F00003620023436283620C30FFF762F948B92E
:103300000120F2E74FF4C063C361F0E74FF480633C
:10331000C361ECE7FDF7BCF80020E6E708B5002242
:10332000B0F8A410D0F8A000FEF711F808BD08B559
:103330000122B0F8A410D0F8A000FEF708F808BDEC
:1033400038B50446154669B1FFF7E8FFE268D3686F
:1033500043F02003D3606DB1E268D36843F080038B
:10336000D36038BDFFF7E3FFE268D36823F02003A2
:10337000D360F0E7E268D36823F08003D360F0E71E
:1033800008B54FF496730C30FFF74BF908B10020E5
:1033900008BD0120FCE708B501231A460C30FFF7F1
:1033A000A6F908B1002008BD0120FCE708B5024BD2
:1033B0001B68984708BD00BF2805002008B5024BD0
:1033C0001B68984708BD00BF2405002084B001A8F1
:1033D00080E80E00012004B07047436D6FF00102D9
:1033E0001A61426DD36843F00103D360436D00223C
:1033F0005A62426D136843F0010313607047436DD6
:10340000196A41F21112114208D1196A40F244427C
:10341000114203D11A6822F001021A60436D0022A2
:103420005A62426DD36823F00103D360436D6FF09D
:1034300001021A617047000008B5024B1B689847EB
:1034400008BD00BF2C050020EFF305837BB9EFF327
:10345000108313B9EFF311831BB1094B1B68022BC7
:1034600008D0074B186840B901221A6070476FF006
:10347000050070476FF0050070474FF0FF30704750
:103480009407002008B5EFF30583A3B9EFF3108389
:1034900013B9EFF311831BB10B4B1B68022B0DD03B
:1034A000094B1B68012B0CD1074B02221A6001F05B
:1034B000FDFA002008BD6FF00500FBE76FF0050086
:1034C000F8E74FF0FF30F5E79407002008B5EFF379
:1034D000058393B9EFF3108313B9EFF311831BB195
:1034E0000B4B1B68022B0BD001F0F2FD58B10228E8
:1034F0000BD101F029FB002009E06FF0050006E088
:103500006FF0050003E0012001E04FF0FF3008BD3F
:103510009407002010B5EFF3058313BB0446EFF3C7
:10352000108313B9EFF311831BB1144B1B68022BEB
:103530001AD001F0CDFD08B1022818D1012C06D017
:10354000C4B901F09BFB012804D1204610BD01F055
:10355000FBFAFAE701F0BCFD0228F6D04FF0FF3489
:10356000F3E76FF00504F0E76FF00504EDE74FF0C7
:10357000FF34EAE74FF0FF34E7E700BF940700208D
:10358000F0B587B000240594EFF30584002C38D102
:10359000EFF3108313B9EFF311831BB12D4B1B68AD
:1035A000022B2ED068B322B31568936903B9182390
:1035B0005C1E372C49D8546814F0010F47D1566966
:1035C0006EB14FEA960C94682CB1D7685B2F02D984
:1035D000176907B1C6B92CB14FF0FF340EE04FF0B8
:1035E000800CF0E7D4688CB9146994B14FF0FF34C3
:1035F00004E01546002418234FF0800C012C0AD05B
:10360000ACB1059807B0F0BD0124F7E74FF0FF34E7
:10361000F4E70024F2E7146992680292019400939F
:103620000B466246294601F0D1F90590E9E705AA63
:10363000019200930B461FFA8CF2294601F001FA21
:103640000128DED000230593DBE70020DAE7002025
:10365000D8E700BF9407002008B5EFF3058383B9CE
:10366000EFF3108313B9EFF311831BB1084B1B6801
:10367000022B09D008B9002008BD01F07BFB002017
:10368000FAE76FF00500F7E76FF00500F4E700BF19
:103690009407002008B5EFF305831BBBEFF31083FD
:1036A00013B9EFF311831BB1114B1B68022B1BD015
:1036B000A0B1836813B1C2681F2A0BD82BB14FF099
:1036C000FF339BB900F0E9F80DE0C36843B14FF058
:1036D000FF33F6E7184600F0BBF804E00023F0E7FC
:1036E0000023EEE7002008BD0020FCE70020FAE7F9
:1036F0009407002070B310B582B00C46034611F059
:103700007F4F2AD1EFF3058272B9EFF3108212B91D
:10371000EFF311821AB1154A1268022A04D0214629
:10372000184600F04CF91AE00022019201AA214645
:10373000184600F08FF9A0B1019BABB14FF0E02328
:103740004FF08052C3F8042DBFF34F8FBFF36F8F3C
:10375000204604E06FF0030070476FF0030002B0F2
:1037600010BD6FF00200FAE72046F8E7940700204A
:1037700090B370B582B00C461D46844611F07F4F61
:103780002DD1EFF3058373BBEFF3108313B9EFF380
:1037900011831BB11A4B1B68022B27D012F00106B4
:1037A00010D0012312F0020F0ED000220095214606
:1037B000604600F080F84EB1844212D0CDB16FF077
:1037C00001000EE00023EDE70122EFE7044208D1FB
:1037D00095B16FF0010004E06FF0030070476FF0E7
:1037E000030002B070BD6FF00500FAE76FF005004E
:1037F000F7E76FF00200F4E76FF00200F1E700BFB7
:1038000094070020034B0360034B0B60802313607D
:10381000704700BF3807002038050020034B0360C5
:10382000034B0B604FF4807313607047980B0020BC
:10383000980700201AB9084206D11046704731EAAD
:10384000000303D00020704701207047012070471B
:1038500080B110B582B0044620230193019B202B38
:1038600011D04FF0500383F31188BFF36F8FBFF374
:103870004F8FFEE74FF0500383F31188BFF36F8F34
:10388000BFF34F8FFEE7002340F8043B00F0ECF855
:1038900001232377204602B010BD38B5202000F068
:1038A000FBFA044628B1002540F8045B00F0DCF880
:1038B0002577204638BD2DE9F84378B10C461646E9
:1038C0001D46074611F07F4811D04FF0500383F397
:1038D0001188BFF36F8FBFF34F8FFEE74FF0500398
:1038E00083F31188BFF36F8FBFF34F8FFEE741B9AA
:1038F0004FF0500383F31188BFF36F8FBFF34F8FE7
:10390000FEE701F0E5FB50B9089B43B14FF05003CF
:1039100083F31188BFF36F8FBFF34F8FFEE701F082
:1039200013F9D7F800902A4621464846FFF782FF50
:10393000F0B116B129EA04033B6001F09FF9B8F138
:10394000000F12D048B94FF0E0234FF08052C3F877
:10395000042DBFF34F8FBFF36F8F01F011FC814631
:1039600010F0007F1AD029F07F494846BDE8F8835F
:10397000089B83B166B941460DB141F08061089A58
:103980002143381D01F07EFAC146DDF82080D4E7DE
:103990004FF08071F0E7DDF82080CEE700F002F90B
:1039A000D7F800902A4621464846FFF743FF18B152
:1039B00016B129EA04043C6000F016F9D3E7F8B523
:1039C00068B10D46044611F07F4711D04FF0500307
:1039D00083F31188BFF36F8FBFF34F8FFEE74FF074
:1039E000500383F31188BFF36F8FBFF34F8FFEE750
:1039F00000F10C0601F0A8F8206923682B4323602E
:103A00000AE0216832EA010105D111E0216841F0A4
:103A1000007101F0C5FA2846B0420ED0456803682F
:103A200023F07F4213F0806FEBD121681142F2D076
:103A300013F0807FEAD01743E8E7236823EA0703FF
:103A4000236001F01BF92068F8BD08B5FFF7B7FF48
:103A500008BD000008B513460A460146014801F0BA
:103A6000C5FD08BD4B3A000800F1080343604FF064
:103A7000FF328260C360036100230360704700234C
:103A80000361704743684B609A688A60516099602F
:103A90000861036801330360704730B40D68B5F105
:103AA000FF3F11D000F108031C465B681A68AA4268
:103AB000FAD963684B6099608C6061600861036843
:103AC0000133036030BC70470469F2E70369416861
:103AD00082688A60416851605A68824206D000223A
:103AE00002611A68013A1A601868704782685A6061
:103AF000F5E7000082B0002301930D4B1B68B3F182
:103B0000FF3F08D04FF0500383F31188BFF36F8F4E
:103B1000BFF34F8FFEE74FF0500383F31188BFF3DD
:103B20006F8FBFF34F8F019B002BFCD002B070470B
:103B3000F400002006480068006880F3088862B638
:103B400061B6BFF34F8FBFF36F8F00DF00BF000080
:103B500008ED00E04FF0807340F8043C21F00101D3
:103B600040F8081C034B40F80C3C40F8202C40382F
:103B7000704700BFF53A0008000000000000000098
:103B8000074B19680868B0E8F00F80F30988BFF3A5
:103B90006F8F4FF0000080F311884EF00D0E7047CC
:103BA0005C1800204FF0500383F31188BFF36F8F30
:103BB000BFF34F8F0B4A136801331360012B00D002
:103BC00070474FF0E023D3F8043D13F0FF0FF7D018
:103BD0004FF0500383F31188BFF36F8FBFF34F8F04
:103BE000FEE700BFF4000020094B1B6843B94FF00B
:103BF000500383F31188BFF36F8FBFF34F8FFEE73E
:103C0000013B034A13600BB983F31188704700BF6F
:103C1000F400002000000000000000000000000090
:103C2000EFF30980BFF36F8F0D4B1A6820E9F00F97
:103C300010602DE908404FF0500080F3118801F02A
:103C4000BFF84FF0000080F31188BDE80840196804
:103C50000868B0E8F00F80F30988BFF36F8F7047F2
:103C60005C18002008B54FF0500383F31188BFF3B0
:103C70006F8FBFF34F8F00F075FF28B14FF0E02337
:103C80004FF08052C3F8042D002383F3118808BD40
:103C90004FF0E022002313619361054B1B68054937
:103CA000A1FB03139B09013B536107231361704779
:103CB00064000020D34D621010B582B02A4B1A78F0
:103CC000D2B20192FF221A701B78DBB28DF803305A
:103CD0009DF8033003F05003244A1370244B07224D
:103CE0001A6009E0224A1368013B13609DF8033013
:103CF0005B00DBB28DF803309DF8033013F0800FCA
:103D0000F0D11B4B1B68032B08D04FF0500383F3FB
:103D10001188BFF36F8FBFF34F8FFEE71B02144A6A
:103D2000136003F4E0631360019BDBB20E4A13706F
:103D30004FF0E023D3F8202D42F47002C3F8202D79
:103D4000D3F8202D42F07042C3F8202DFFF7A0FFDA
:103D50000024084B1C60FFF7EDFE01F031F8FFF77F
:103D6000C9FE204602B010BD00E400E0F40B0020C4
:103D7000F80B0020F4000020EFF305830F2B0FD980
:103D8000114A9B5CDBB2114A12789A4208D94FF073
:103D9000500383F31188BFF36F8FBFF34F8FFEE79C
:103DA0004FF0E023D3F80C3D03F4E063084A1268B7
:103DB000934208D94FF0500383F31188BFF36F8FFC
:103DC000BFF34F8FFEE77047F0E300E0F40B0020F5
:103DD000F80B0020124A12F0070F1ED0D11D21F05F
:103DE0000701C1F5406313440A460E4802600021F2
:103DF00041601344083B23F007030B4803605960FC
:103E00001960991A51601360084B1960084B1960CA
:103E1000084B4FF000421A6070474FF44063E4E7EC
:103E2000000C002014180020FC0B002008180020B3
:103E30000418002000180020154B1A461B68834206
:103E4000FBD3516802EB010C844509D0416800EBBB
:103E5000010C634509D00360904218D01060704790
:103E60004068014451601046F0E710B4094C2468E2
:103E7000A3420AD05B681944416013681B68036061
:103E8000904200D0106010BC70470460F8E77047A3
:103E900014180020FC0B002070B5054600F054FEFD
:103EA000364B1B68A3B1364B1B681D424ED135B152
:103EB000083515F0070F02D025F007050835002D4D
:103EC00046D0304B1B68AB4251D32F4A146804E0F4
:103ED000FFF780FFE7E722461C466368AB4202D249
:103EE0002368002BF7D1254B1B68A34241D01668ED
:103EF00008362368136063685B1B102B10D96019A8
:103F000010F0070F08D04FF0500383F31188BFF370
:103F10006F8FBFF34F8FFEE743606560FFF78CFF45
:103F2000626818490B689B1A0B60184909688B4234
:103F300001D216490B60124B1B68134363600023C8
:103F40002360134A13680133136002E0002600E087
:103F5000002600F093FE16F0070F0CD04FF0500330
:103F600083F31188BFF36F8FBFF34F8FFEE70026F7
:103F7000EFE70026EDE7304670BD00BFFC0B0020E8
:103F80000018002004180020141800200818002031
:103F90000C180020002834D038B50446A0F10805DC
:103FA00050F8043C174A1268134208D14FF05003EE
:103FB00083F31188BFF36F8FBFF34F8FFEE750F885
:103FC000081C41B14FF0500383F31188BFF36F8F8A
:103FD000BFF34F8FFEE723EA020340F8043C00F0F2
:103FE000B3FD54F8041C084A13680B4413602846B8
:103FF000FFF722FF054A13680133136000F03EFE0D
:1040000038BD704700180020041800201018002048
:1040100010B50446FFF7C6FDA26BE36B9A4204D0CD
:104020000024FFF7E1FD204610BD0124F9E710B59B
:104030000446FFF7B7FDA36B23B90124FFF7D4FDB6
:10404000204610BD0024F9E770B504461546866B7E
:10405000026C5AB903681BB100200136A66370BD1B
:10406000806801F045F80023A360F6E76DB9406869
:10407000FCF7BEF8226C636813446360A268934245
:1040800019D3236863602846E7E7C068FCF7B0F8F7
:10409000226C5142E3689B1AE3602268934202D289
:1040A000A3680B44E360022D01D00020D5E726B1C0
:1040B000013E0020D1E72846CFE70020CDE708B534
:1040C0000346026C62B10846D9681144D960D3F83E
:1040D00008C0614501D31968D960D968FCF788F830
:1040E00008BD38B50546FFF75DFD95F8454064B25B
:1040F00001E0013C64B2002C0ADD6B6A43B105F1BA
:10410000240000F007FF0028F3D000F0DBFFF0E709
:10411000FF2385F84530FFF767FDFFF743FD95F86E
:10412000444064B201E0013C64B2002C0ADD2B691A
:1041300043B105F1100000F0EDFE0028F3D000F0CF
:10414000C1FFF0E7FF2385F84430FFF74DFD38BD90
:1041500038B5E0B10D460446FFF724FD2368E26B55
:10416000216C01FB0230A0600020A0636360013A73
:1041700002FB0133E360FF2384F8443084F84530C8
:10418000FDB9236963B9FFF72FFD012038BD4FF05A
:10419000500383F31188BFF36F8FBFF34F8FFEE798
:1041A00004F1100000F0B6FE0028ECD04FF0E02340
:1041B0004FF08052C3F8042DBFF34F8FBFF36F8FC2
:1041C000E1E704F11000FFF74FFC04F12400FFF7D2
:1041D0004BFCD8E738B51D46049C0B4649B9246012
:1041E000E063236401212046FFF7B2FF84F84C50BE
:1041F00038BD2260F4E740B94FF0500383F31188D3
:10420000BFF36F8FBFF34F8FFEE710B584B01C462E
:10421000844653B192B189B94FF0500383F31188AA
:10422000BFF36F8FBFF34F8FFEE74FF0500383F361
:104230001188BFF36F8FBFF34F8FFEE76AB1502332
:104240000393039B502B13D04FF0500383F311883B
:10425000BFF36F8FBFF34F8FFEE70029EFD04FF012
:10426000500383F31188BFF36F8FBFF34F8FFEE7C7
:10427000039B012384F8463000949DF81830604673
:10428000FFF7A8FF204604B010BDF0B585B001923D
:1042900088B10F461D460446B1B1022D20D1E36B13
:1042A000012B1DD04FF0500383F31188BFF36F8FA4
:1042B000BFF34F8FFEE74FF0500383F31188BFF336
:1042C0006F8FBFF34F8FFEE7036C002BE5D04FF0ED
:1042D000500383F31188BFF36F8FBFF34F8FFEE757
:1042E00000F0F6FE064658B9019B002B48D04FF06F
:1042F000500383F31188BFF36F8FBFF34F8FFEE737
:1043000000263DE02A4639462046FFF79DFE636AB7
:104310007BB948B14FF0E0234FF08052C3F8042D31
:10432000BFF34F8FBFF36F8FFFF75EFC012005B027
:10433000F0BD04F1240000F0EDFD0028F4D04FF0B2
:10434000E0234FF08052C3F8042DBFF34F8FBFF32B
:104350006F8FE9E7FFF748FC0020E8E702A800F0CC
:1043600063FE012619E0002384F8443021E0002395
:1043700084F8453023E02046FFF7B3FE00F07EFCD2
:10438000FFF710FCA26BE36B9A42BBD3022DB9D0AE
:10439000019B002BDED0002EE0D0FFF725FC00F0C3
:1043A000D3FBFFF7FFFB94F8442052B2B2F1FF3F7A
:1043B000D9D094F8452052B2B2F1FF3FD7D0FFF7E1
:1043C00013FC01A902A800F03BFED8B92046FFF774
:1043D0001FFE0028CFD0019904F1100000F03AFD33
:1043E0002046FFF77EFE00F049FC0028C8D14FF0C0
:1043F000E0234FF08052C3F8042DBFF34F8FBFF37B
:104400006F8FBDE72046FFF76CFE00F037FC002001
:104410008DE72DE9F84390B10F4616461C46054638
:10442000B1B1022C20D1EB6B012B1DD04FF050030A
:1044300083F31188BFF36F8FBFF34F8FFEE74FF009
:10444000500383F31188BFF36F8FBFF34F8FFEE7E5
:10445000036C002BE5D04FF0500383F31188BFF3BA
:104460006F8FBFF34F8FFEE7FFF786FCEFF31189E5
:104470004FF0500383F31188BFF36F8FBFF34F8F5B
:10448000AA6BEB6B9A4206D3022C04D0002089F36E
:104490001188BDE8F88395F845804FFA88F8AB6B32
:1044A000224639462846FFF7CFFDB8F1FF3F06D038
:1044B00008F101035BB285F845300120E7E76B6A3C
:1044C0000BB90120E3E705F1240000F023FD18B14A
:1044D00026B101203060DAE70120D8E70120D6E7D5
:1044E000F0B585B0019290B10F460446C1B100F01D
:1044F000EFFD064600BB019B002B5ED04FF0500342
:1045000083F31188BFF36F8FBFF34F8FFEE74FF038
:10451000500383F31188BFF36F8FBFF34F8FFEE714
:10452000036C002BE3D04FF0500383F31188BFF3EB
:104530006F8FBFF34F8FFEE700263EE039462046DF
:10454000FFF7BDFD013DA563236923B9FFF74CFBD0
:10455000012005B0F0BD04F1100000F0DBFC0028E4
:10456000F4D04FF0E0234FF08052C3F8042DBFF396
:104570004F8FBFF36F8FE9E7FFF736FB0020E8E7C7
:1045800002A800F051FD012621E0002384F8443008
:1045900029E0002384F845302BE02046FFF7A1FDF9
:1045A00000F06CFB09E02046FFF79BFD00F066FB86
:1045B0002046FFF73CFD00283FD1FFF7F3FAA56B3B
:1045C000002DBBD1019B002BD6D0002ED8D0FFF7F9
:1045D0000BFB00F0B9FAFFF7E5FA94F844305BB250
:1045E000B3F1FF3FD1D094F845305BB2B3F1FF3F58
:1045F000CFD0FFF7F9FA01A902A800F021FD0028A9
:10460000D1D12046FFF713FD0028C6D0019904F14F
:10461000240000F01FFC2046FFF763FD00F02EFB96
:104620000028CAD14FF0E0234FF08052C3F8042D88
:10463000BFF34F8FBFF36F8FBFE7002089E7000004
:104640000023072B0CD8074A52F833200AB1013354
:10465000F7E7044A42F8331002EBC303586070478F
:10466000704700BF1C18002070B504460D46164662
:10467000FFF798FA94F844305BB2B3F1FF3F0DD0E6
:1046800094F845305BB2B3F1FF3F0BD0FFF7ACFAC3
:10469000A36B5BB12046FFF724FD70BD002384F8B7
:1046A0004430EDE7002384F84530EFE732462946F1
:1046B00004F1240000F012FCECE70000084B1B683A
:1046C0001B6823B9074B4FF0FF321A607047044B49
:1046D0001B68DB68DB685A68024B1A60704700BFD2
:1046E00060180020081D00202DE9F04780460D4687
:1046F00017469946089EDDF824A00A9C9200A52141
:10470000206B00F0ABFF236B07F18042013A03EB13
:10471000820727F00707B5B34FF0000CBCF10F0F6D
:104720000BD815F80C2004EB0C0383F8342015F893
:104730000C3013B10CF1010CF0E7002384F8433086
:10474000372E00D93726E662E66400252565201D50
:10475000FFF795F904F11800FFF791F92461C6F10C
:104760003806A6616462656584F858504A46414639
:104770003846FFF7EFF92060BAF1000F01D0CAF810
:104780000040BDE8F087002384F83430D8E700000B
:1047900038B5002407E004EB840293000E48184467
:1047A000FFF762F90134372CF5D90C4D2846FFF795
:1047B0005BF90B4C2046FFF757F90A48FFF754F90D
:1047C0000948FFF751F90948FFF74EF9084B1D60FA
:1047D000084B1C6038BD00BF68180020DC1C00209E
:1047E000F01C0020141D0020401D00202C1D002066
:1047F000601800206418002010B50446FFF7D2F9B5
:10480000224A136801331360214B1B685BB1214BB3
:104810001B686BB91E4B1B68DA6AE36A9A4207D8B9
:104820001B4B1C6004E01A4B1C601368012B29D041
:10483000194A1368013313606364E06A174B1B68FD
:10484000984201D9154B186000EB8000211D144BD4
:1048500003EB8000FFF716F9FFF7C6F90D4B1B6855
:104860007BB10B4B1B68DA6AE36A9A4209D24FF0BC
:10487000E0234FF08052C3F8042DBFF34F8FBFF3F6
:104880006F8F10BDFFF784FFD2E700BFC81C002068
:104890005C180020281D0020D41C0020D81C0020FB
:1048A0006818002010B5044690F8593063B1012B08
:1048B00011D0022B0ED04FF0500383F31188BFF3B9
:1048C0006F8FBFF34F8FFEE7006BFFF763FB204650
:1048D000FFF760FB10BDFFF75DFBFBE70F4B1B68AD
:1048E000D3B110B5FFF75EF90D4BDB68DC68201D16
:1048F000FFF7ECF80B4A1368013B1360074A136893
:10490000013B1360FFF770F92046FFF7CBFF034B25
:104910001B68002BE6D110BD704700BFCC1C0020E7
:10492000401D0020C81C002008B5FFF7D7FF074B2B
:104930001B68012BF9D94FF0E0234FF08052C3F8E8
:10494000042DBFF34F8FBFF36F8FEEE76818002081
:1049500070B504460D46174B1E68174B1868043097
:10496000FFF7B4F8B4F1FF3F0DD03444124B1B688D
:104970005C60A64210D9114B18680F4B19680431BE
:10498000FFF78BF870BD002DEFD00B4B1968043189
:104990000B48FFF777F8F5E70A4B1868064B1968DC
:1049A0000431FFF77AF8084B1B68A342EAD9064B9B
:1049B0001C60E7E7541D00205C18002064180020EC
:1049C0002C1D002060180020081D002030B587B085
:1049D0000B9C7CB10C9DB5B15C250495049D5C2DB0
:1049E0001AD04FF0500383F31188BFF36F8FBFF3DA
:1049F0004F8FFEE74FF0500383F31188BFF36F8FA3
:104A0000BFF34F8FFEE74FF0500383F31188BFF3DE
:104A10006F8FBFF34F8FFEE7049D0C9D2C63022424
:104A200085F8594000240394029505AC01940A9C32
:104A30000094FFF759FE0C98FFF7DEFE059807B0CB
:104A400030BD2DE9F04385B00746884614461E4622
:104A50009000FFF721FA00B381465C20FFF71CFAB3
:104A60000546B0B1C0F83090E5B1002385F8593063
:104A7000039302950D9B01930C9B009333462246B2
:104A800041463846FFF730FE2846FFF7B5FE0120C5
:104A900005E04846FFF77EFAE6E74FF0FF3005B045
:104AA000BDE8F0834FF0FF30F9E7000010B588B0A3
:104AB00000240594069407AA06A905A8FEF7A2FEFD
:104AC000059B0293069B019300942346079A18497D
:104AD0001848FFF77BFF184B186040B100F0C8FB87
:104AE000012806D0B0F1FF3F18D008B010BD00205B
:104AF000F6E74FF0500383F31188BFF36F8FBFF3D6
:104B00004F8F0E4B4FF0FF321A600D4B01221A608F
:104B10000C4B00221A60FFF7CFF8E6E74FF0500386
:104B200083F31188BFF36F8FBFF34F8FFEE700BF92
:104B30008059000829490008041D0020081D002094
:104B4000281D0020541D0020024A13680133136001
:104B5000704700BFD01C0020014B1868704700BF91
:104B6000541D0020F8B53A4B1B68002B69D1394B16
:104B70001D6801351D60C5B9374B1B681B6843B103
:104B80004FF0500383F31188BFF36F8FBFF34F8F44
:104B9000FEE7314A1168314B186810601960304ADD
:104BA000136801331360FFF789FD2E4B1B68AB427E
:104BB0003DD900272C4B1B68DB6A03EB83039A006B
:104BC0002A4B9B58012B00D90127294B1B68002B2E
:104BD0003CD001273AE001271F4B1B681B6843B3F9
:104BE0001D4B1B68DB68DC6863689D4226D3261D6D
:104BF0003046FEF76BFFA36A1BB104F11800FEF705
:104C000065FFE36A1B4A1268934201D9194A13608F
:104C100003EB83039A00314614481044FEF732FF39
:104C2000E26A114B1B68DB6A9A42D4D2D4E70027B0
:104C3000D2E70C4B4FF0FF321A60BBE7094A136012
:104C4000B8E70D4A13680133136000273846F8BDF2
:104C5000D01C0020541D0020601800206418002083
:104C60000C1D0020081D00205C1800206818002082
:104C7000581D0020D81C0020101D002038B5354BD1
:104C80001B6843B94FF0500383F31188BFF36F8F54
:104C9000BFF34F8FFEE7FEF785FF2E4B1A68013AF0
:104CA0001A601B68002B4FD12B4B1B680BB90024DB
:104CB0004BE00024294B1B681BB3284BDB68DC68E6
:104CC00004F11800FEF702FF251D2846FEF7FEFE40
:104CD000E06A234B1B68984201D9214B186000EB16
:104CE000800029461F4B03EB8000FEF7CBFEE26AF3
:104CF0001D4B1B68DB6A9A42DCD31C4B01221A60F5
:104D0000D8E70CB1FFF7DAFC194B1C6884B9174BD4
:104D10001C68D4B14FF0E0234FF08052C3F8042D4B
:104D2000BFF34F8FBFF36F8F01240EE0013C07D01C
:104D3000FFF718FF0028F9D00C4B01221A60F5E7A5
:104D40000B4B00221A60E2E70024FEF74DFF2046DD
:104D500038BD00BFD01C0020C81C0020141D00203E
:104D6000D81C0020681800205C180020581D002066
:104D7000101D002010B5A8B10446104B1B6843B1AC
:104D80004FF0500383F31188BFF36F8FBFF34F8F42
:104D9000FEE7FFF7D9FE00212046FFF7D9FDFFF718
:104DA0006DFF48B94FF0E0234FF08052C3F8042D57
:104DB000BFF34F8FBFF36F8F10BD00BFD01C00201B
:104DC0001F4B1B681BB11F4B01221A6070471D4B04
:104DD00000221A601C4B1B6803EB83018A001B49ED
:104DE0008A585AB90BB1013BF6E74FF0500383F3F1
:104DF0001188BFF36F8FBFF34F8FFEE703EB830084
:104E000082000A4450684068506003EB830C4FEA0C
:104E10008C020832114488420BD003EB83029100CC
:104E20000A4A0A445268D168094A1160064A136066
:104E30007047406862469100044A0A445060ECE7BB
:104E4000D01C0020581D0020D81C0020681800200D
:104E50005C18002058B110B50C46094A1168183189
:104E6000FEF71BFE01212046FFF772FD10BD4FF03B
:104E7000500383F31188BFF36F8FBFF34F8FFEE7AB
:104E80005C18002070B110B514460246114B1B6827
:104E90008BB94FF0500383F31188BFF36F8FBFF3CB
:104EA0004F8FFEE74FF0500383F31188BFF36F8FEE
:104EB000BFF34F8FFEE7084B186841F00041816156
:104EC000196818311046FEF7DDFD01212046FFF775
:104ED0003FFD10BDD01C00205C18002038B570B11B
:104EE0000D4614460A4A11681831FEF7CBFD0CB185
:104EF0004FF0FF3521462846FFF72AFD38BD4FF019
:104F0000500383F31188BFF36F8FBFF34F8FFEE71A
:104F10005C18002038B5C368DC6824B304F11805B8
:104F20002846FEF7D3FD184B1B682BBB251D2846D2
:104F3000FEF7CCFDE06A154B1B68984201D9134B74
:104F4000186000EB80002946114B03EB8000FEF750
:104F500099FDE26A0F4B1B68DB6A9A4211D9012066
:104F60000D4B186038BD4FF0500383F31188BFF329
:104F70006F8FBFF34F8FFEE729460848FEF782FD8B
:104F8000E7E70020EEE700BFD01C0020D81C00207F
:104F9000681800205C180020581D0020141D0020F7
:104FA00038B51C4B1B6843B94FF0500383F311888D
:104FB000BFF36F8FBFF34F8FFEE741F000410160F9
:104FC000C468F4B1FEF782FD251D2846FEF77EFD7C
:104FD000E06A114B1B68984201D90F4B186000EB37
:104FE000800029460D4B03EB8000FEF74BFDE26A83
:104FF0000B4B1B68DB6A9A4202D90A4B01221A60EA
:1050000038BD4FF0500383F31188BFF36F8FBFF3A8
:105010004F8FFEE7D01C0020D81C0020681800200D
:105020005C180020581D0020034B1B680360034BD5
:105030001B684360704700BF0C1D0020541D0020FA
:10504000D8B170B50C46054601B3FEF7ABFD1B4B5E
:1050500019686B68C81A2268B2F1FF3F27D0184E52
:105060003668D5F800C0B44501D08B4224D98242BD
:1050700015D80023236001241AE04FF0500383F376
:105080001188BFF36F8FBFF34F8FFEE74FF05003D0
:1050900083F31188BFF36F8FBFF34F8FFEE75B1A67
:1050A000134423602846FFF7BFFF002400E00024DC
:1050B000FEF79AFD204670BD0124F9E7541D00203B
:1050C0000C1D0020014B01221A607047581D002062
:1050D000054B1B6833B1054B1B680BB100207047B3
:1050E0000220704701207047281D0020D01C00209E
:1050F00000283BD038B504461E4B1B68834208D0BD
:105100004FF0500383F31188BFF36F8FBFF34F8FBE
:10511000FEE7036D43B94FF0500383F31188BFF3EB
:105120006F8FBFF34F8FFEE7013B0365C16AC26C0F
:1051300091421DD00BB1002038BD051D2846FEF759
:10514000C5FCE06CE062C0F13803A3610A4B1B6848
:10515000984201D9084B186000EB80002946074BA4
:1051600003EB8000FEF78EFC0120E5E7002070478E
:105170000020E1E75C180020D81C002068180020FF
:10518000044A136898691368DB6A1268C3F138032C
:10519000936170475C180020064B1A6813682BB99E
:1051A0000123036023B9D368186870470023F8E728
:1051B000002070475C1D002008B5416000619142ED
:1051C0000CD8D21A83699A4201D3012008BD011D6F
:1051D000094B1868FEF761FC0020F7E79A4201D2FC
:1051E000994206D2011D054B1868FEF756FC0020B7
:1051F000ECE70120EAE700BF601D00205C1D0020F5
:1052000030B583B0FEF7CEFC114B1B681BB1FEF727
:10521000EBFC03B030BD0F4D2846FEF725FC0E4CCD
:105220002046FEF721FC0D4B1D600D4B1C6000233A
:1052300000930C4B0C4A10210A20FEF7DCFF044BB4
:1052400018600028E3D00949FFF7FAF9DFE700BF4B
:10525000801E0020041E0020181E00205C1D00205F
:10526000601D0020301E0020641D002088590008A9
:1052700010B588B0FFF7C4FF124B1B68CBB10024F8
:105280000594069407AA06A905A8FEF7C7FA059B88
:105290000293069B0193022300932346079A0A492F
:1052A0000A48FFF793FB0A4B186010B1012008B0C1
:1052B00010BD4FF0500383F31188BFF36F8FBFF31E
:1052C0004F8FFEE7801E002090590008D55500083A
:1052D000841E0020B8B19C4603461848006858B3A5
:1052E00000B585B000910192029305291CDCFFF7FF
:1052F000EFFE022810D000231A4669460F480068C6
:10530000FEF7C3FF15E04FF0500383F31188BFF39E
:105310006F8FBFF34F8FFEE70023069A6946074859
:105320000068FEF7B2FF04E0002362466946FFF71B
:1053300070F805B05DF804FB00207047801E002067
:1053400070B582B01B4B1B681A6862B3DB681E68BD
:10535000DC68251D2846FEF7B9FB236A20469847DE
:1053600094F8283013F0040FECD0A36933449E4224
:1053700007D26360246129460E4B1868FEF78DFB47
:10538000E0E7002100910B4632462046FFF7A2FFDE
:105390000028D7D14FF0500383F31188BFF36F8FEC
:1053A000BFF34F8FFEE7044A10680249086013609C
:1053B00002B070BD5C1D0020601D002038B50546A0
:1053C000FFF7CAFB0446074B1B68834205D800233E
:1053D0002B60044B1C60204638BDFFF7B1FF012352
:1053E0002B60F6E72C1E002070B582B006460D46F5
:1053F00017490968C968CC68201DFEF767FB94F857
:1054000028C01CF0040F08D12CF0010C84F828C02F
:10541000236A2046984702B070BDA16933462A46E8
:1054200031442046FFF7C8FE0028F1D0002100914A
:105430000B4632462046FFF74DFF0028E8D14FF0DB
:10544000500383F31188BFF36F8FBFF34F8FFEE7D5
:105450005C1D002070B582B006460C46FFF774FB59
:1054600001A8FFF7ABFF019B33BB05460CB9B04267
:1054700019D224B1124A12681268DAB901242246FC
:10548000711B104B1868FFF7EFF8FFF7F7FBA8B98F
:105490004FF0E0234FF08052C3F8042DBFF34F8F3D
:1054A000BFF36F8F0AE0FFF7E9FB29463046FFF7AD
:1054B0009BFF03E01C46E2E7FFF7E0FB02B070BD94
:1054C000601D0020801E002010B588B002E0049B03
:1054D000002B0FDA002204A93D4B1868FFF700F8F3
:1054E000002873D0049B002BF1DA07990698059BDE
:1054F0009847ECE7069C636913B1201DFEF7E6FAB6
:1055000003A8FFF75BFF049B092BE3D8DFE803F058
:105510000505053037500505303794F8283043F03D
:10552000010384F82830059BA169024619442046EE
:10553000FFF742FE0028CDD0236A2046984794F812
:10554000283013F0040FC5D0A269002100910B464A
:10555000059802442046FFF7BDFE0028BAD14FF05F
:10556000500383F31188BFF36F8FBFF34F8FFEE7B4
:1055700094F8283023F0010384F82830AAE794F83F
:10558000283043F0010384F828300599A16131B136
:105590000346024601442046FFF70EFE9AE74FF00D
:1055A000500383F31188BFF36F8FBFF34F8FFEE774
:1055B00094F8283013F0020F04D023F0010384F88C
:1055C000283087E72046FEF7E5FC83E708B010BDEA
:1055D000801E002000B583B001A8FFF7DDFD019912
:1055E000FFF738FFFFF770FFF6E7000010B584B053
:1055F00014461A466FF00103009301900291039440
:105600000023694602480068FEF703FF04B010BD9E
:10561000801E002070B50D4E0D4D761BB61006D0C5
:10562000002455F8043B01349847A642F9D1094EAD
:10563000094D00F065F8761BB61006D0002455F829
:10564000043B01349847A642F9D170BD0000000028
:10565000000000000000000000000000830730B5DB
:1056600048D0541E002A3FD00346CAB201E0013C94
:105670003AD303F8012B9D07F9D1032C2DD9CDB2D4
:1056800045EA05250F2C45EA054536D9A4F1100257
:1056900022F00F0C03F1200EE6444FEA121C03F136
:1056A000100242E9045542E9025510327245F8D120
:1056B0000CF1010214F00C0F03EB021204F00F0CBA
:1056C00013D0ACF1040323F003030433134442F872
:1056D000045B9342FBD10CF003042CB1CAB21C440E
:1056E00003F8012B9C42FBD130BD64461346002CCD
:1056F000F4D1F9E703461446BFE71A46A446E0E7AB
:10570000F8B500BFF8BC08BC9E467047F8B500BFAE
:08571000F8BC08BC9E4670477E
:1057180064656661756C745461736B001857000892
:105728000000000000000000000000000000000071
:105738000002000018000000000000000000000047
:10574800736C6176655F3438350000000000000036
:105758000000000001020304060708090000000019
:105768000102030402030405060708090A0B0C0DCD
:105778000E0F10100102000000C1814001C08041DD
:1057880001C0804100C1814001C0804100C1814009
:1057980000C1814001C0804101C0804100C18140F9
:1057A80000C1814001C0804100C1814001C08041E9
:1057B80001C0804100C1814001C0804100C18140D9
:1057C80000C1814001C0804100C1814001C08041C9
:1057D80001C0804100C1814000C1814001C08041B9
:1057E80001C0804100C1814001C0804100C18140A9
:1057F80000C1814001C0804101C0804100C1814099
:1058080000C1814001C0804100C1814001C0804188
:1058180001C0804100C1814000C1814001C0804178
:1058280001C0804100C1814001C0804100C1814068
:1058380000C1814001C0804100C1814001C0804158
:1058480001C0804100C1814001C0804100C1814048
:1058580000C1814001C0804101C0804100C1814038
:1058680000C1814001C0804100C1814001C0804128
:1058780001C0804100C1814000C0C101C30302C210
:10588800C60607C705C5C404CC0C0DCD0FCFCE0E78
:105898000ACACB0BC90908C8D81819D91BDBDA1AE8
:1058A8001EDEDF1FDD1D1CDC14D4D515D71716D658
:1058B800D21213D311D1D010F03031F133F3F232C8
:1058C80036F6F737F53534F43CFCFD3DFF3F3EFE38
:1058D800FA3A3BFB39F9F83828E8E929EB2B2AEAA8
:1058E800EE2E2FEF2DEDEC2CE42425E527E7E62618
:1058F80022E2E323E12120E0A06061A163A3A26288
:1059080066A6A767A56564A46CACAD6DAF6F6EAEF7
:10591800AA6A6BAB69A9A86878B8B979BB7B7ABA67
:10592800BE7E7FBF7DBDBC7CB47475B577B7B676D7
:1059380072B2B373B17170B0509091519353529247
:1059480096565797559594549C5C5D9D5F9F9E5EB7
:105958005A9A9B5B99595898884849894B8B8A4A27
:105968004E8E8F4F8D4D4C8C448485458747468697
:10597800824243834181804049444C4500000000F5
:10598800546D725100000000546D7220537663000C
:1059980000000000C803002004000000C803002025
:1059A80008000000C8030020000C0140200000008F
:1059B800000C014040000000000C01408000000085
:1059C800000C014000010000000C01400002000032
:1059D8004857000800000000000000000000000018
:1059E800000000000003000020000000000000008C
:1059F8000000000000127A00010000001000000002
:105A08000200000011000000352D0008030000000E
:105A18000D2C000810000000AD2B00080600000047
:105A2800792B0008170000007D2C000814000000E6
:105A3800612B0008000000000000000000000000CA
:105A4800000000000000000000000000000000004E
:105A5800000000000000000000000000000000003E
:105A6800000000000000000000000000000000002E
:105A7800000000000000000000000000000000001E
:085A880000000000AAAAAAAA6E
:0400000508000DEDF5
:00000001FF
